:020000040000FA
:0400000016EF00F007
:08000800006ED8CF02F0E0CF3A
:1000100001F0F2B2F7EC00F09EB0E3EC00F000D09B
:1000200001C0E0FF005002C0D8FF1000806A816A62
:10003000826A0F0EC16E070EB46E000E946E2A6AAD
:100040002B6A800E096E0A6E0B6E0C6E0D6E0E6EB4
:100050000F6E106E46EC01F0C80ED56E9E0E046E4B
:10006000580E036EB40ECD6E0450CF6E0350CE6E9C
:100070009E909D80EEEC00F0CD80E80E066EF00EB6
:10008000056E800EB16ED09EF28EF28C2C6A0650F8
:10009000196E1A6E1B6E1C6E1D6E1E6E1F6E206E0C
:1000A0000550116E126E136E146E156E166E176E6D
:1000B000186EC80E216E226E236E246E256E266E7B
:1000C000276E286E2B9010EE09F02BA0FED7CFECF8
:1000D00000F085EC00F0A192B180A1A2FED7E7501C
:1000E000296E20EE21F02A50DBCFD6FFF294F2A445
:1000F000FED7292EF6D7AAEC00F02A28070B2A6E85
:10010000D8B4E0D7E650E3D7C1D7E86A2A6202D074
:1001100082801200E8282A6202D082821200E82837
:100120002A6202D082841200E8282A6202D08286E3
:100130001200E8282A6202D082881200E8282A6287
:1001400002D0828A1200E8282A6202D0828C120031
:10015000828E1200E86A2A6202D082901200E82899
:100160002A6202D082921200E8282A6202D0829487
:100170001200E8282A6202D082961200E8282A6239
:1001800002D082981200E8282A6202D0829A1200D5
:10019000E8282A6202D0829C1200829E1200B1904E
:1001A0000650086E0550076E20EE11F02A50DBCF86
:1001B00007F020EE19F02A50DBCF08F00850B36E9C
:1001C0000750B26E1200CD900450CF6E0350CE6E29
:1001D0009E909D80CD802B80120012009380938290
:1001E000F18CF292F2882E6A080E2F6E1200FCEC4F
:1001F00000F0F292F2881200D89081B2D8803332A7
:100200002E502D6ED8902D36020ED8B0E828FA6EFA
:100210001A0E2D24D8B0FA2AF96E02D00AD016D0C0
:100220002F2E1200010E2E6E060E2F6E3350306EE2
:1002300012002F2E1200020E2E6E080E2F6E33505B
:10024000316ED8903132D890313212002F2E1200F8
:10025000000E2E6E080E2F6E210E306212003350EB
:10026000326E00EE09F0315032C0EBFF12000A0E80
:10027000346E010E366EC80E356E00000000352E4D
:10028000FCD7362EF8D7342EF4D712000A0E346E6F
:10029000FA0E366EC80E356E00000000352EFCD703
:1002A000362EF8D7342EF4D712000A0E346E366E7E
:1002B000C80E356E00000000352EFCD7362EF8D75C
:1002C000342EF5D712000A0E346E010E366E320E41
:1002D000356E00000000352EFCD7362EF8D7342EB0
:1002E000F4D7120046EC01F046EC01F046EC01F0C8
:0602F00046EC01F01200D3
:020000040030CA
:0E000000FF36FEFEFFFDFAFFFFFFFFFFFFFFD2
:00000001FF
